:1000000009298030A100FE30A7200130A7207530DB
:10001000A7003030BF28A101A117AF00AF08031D12
:100020001328030114280130AF020310A20CA20C04
:10003000A20CC0302205403EAF07FE30A7202F089B
:10004000A728A101A117AF00FE30A7202F08A728DD
:10005000A401AA00AB01A01124080319A0150530C2
:10006000A3002730A900103041200330A900E83058
:100070004120A90164304120A9010A3041202A0809
:100080004828A8002B08A7002A08A600D320260885
:10009000A600A3030319A011240803195228230260
:1000A000031859282608031DA011A0195928303E0D
:1000B000A7280800AD0006118611831606118611C7
:1000C0000F30860583122D08A01884283E30A70023
:1000D0008030BF203330AC0098201330A700883028
:1000E000BF2098206430BE2098206430BE2022308B
:1000F000AC009820283083200C30832006308320E9
:10010000A0142D0884282014AC00201C92288611ED
:10011000033C031C972897200730A700D030BF204E
:10012000031408002014FE3C0319A5288615201C82
:10013000201006150F3086052C08F03986040611AC
:10014000AC0E201898283230BE202D080529A11B9E
:100150005A28080083178001840AFF3E031DAB283C
:100160000529A901A800FF30A807031CA907031C43
:1001700005290330A700DF30BF20B328A701E83EE0
:10018000A600A709FC30031CC828A6070318C52829
:10019000A6070000A70FC5282618CE28A61CD2281F
:1001A0000000D2280800AB01AA011030AC00270DD6
:1001B000AA0DAB0D2808AA022908031C290FAB02BF
:1001C0000318E9282808AA0729080318290FAB07EC
:1001D0000310A60DA70DAC0BD72826080529103053
:1001E000B000A701A601AD0CAC0C031CFD2828082B
:1001F000A60729080318290FA707A70CA60CAB0C04
:10020000AA0CB00BF3282A080529831383120313C1
:100210000800A00107309F00E03083168500FF3002
:1002200086008113831285018601203084006030AE
:10023000AB20A03084005030AB2020308400303020
:10024000AA20C830B120012077305A205A205A20E5
:100250002E305A2070305A2069305A2063305A208C
:1002600062305A208030A100C030212061305A20F5
:1002700073305A2069305A2063305A202E305A2069
:100280006E305A206C305A200B30A900B830B220A2
:10029000012044305A2043305A2046305A20313011
:1002A0005A2036305A2055305A204B305A2046308A
:1002B0005A208030A100C230212056305A202D30E3
:1002C0005A2032305A200730A900D030B220012005
:1002D00041305A2064305A206A305A2075305A20F2
:1002E00073305A2074305A2020305A204C305A2013
:1002F0008030A100C030212044305A2052305A2092
:1003000086188829851F86290514872905108029C4
:10031000012053305A2065305A2061305A20723003
:100320005A2063305A2068305A2020305A207330C7
:100330005A208030A100C030212069305A20673017
:100340005A206E305A2061305A206C305A2049149D
:100350008316051283120512392AC2013B03A50038
:10036000C80148082502031CC529E821C91CC22967
:100370004808A200A601A20A0314A60DA20BBD29DB
:100380002608C204C80A031DB1294208B100B201FF
:10039000B20CB10CB20CB10CB20CB10CB20CB10C71
:1003A0000F30B2053108AC003208AD000A30A800A9
:1003B000A901EF20B1002B08B2004208B300B4013C
:1003C0000F30B3050030B40531083307C200080010
:1003D000B801B9010618FD290130B120B80A031986
:1003E000B90A0B303902031CFC29031DFB29B93063
:1003F0003802031CFC295F2CEA299B30B1208310B2
:10040000061883148318C914831CC910491C1C2A9C
:100410004308B100B2010310B10DB20DB10DB20D20
:10042000B10DB20D3108A6003208A7003A30A8007D
:10043000A901D320BC002F2A8030A1000230A200E5
:100440003C080D200230A40043082920030149196B
:10045000013EC918013A03194911031D4915C30A80
:1004600085140130A900F430B2208510F030B1209D
:100470000800BA01C3014912491AD22AB801B901C8
:10048000061C532AB80A0319B90A0130B120AF304B
:100490003902031C522A031D512AC9303802031C99
:1004A000522A5F2C402AB801B90106188F2AB80ACF
:1004B0000319B90A0A30B1204918832A38080B3ABF
:1004C0003904031D6E2A8030A1000230A2003C08CE
:1004D0000D2035305A2039305A20822A3808193AEE
:1004E0003904031D752A8514822A38084B3A3904C9
:1004F000031D7C2A8510822A3808FA3A3904031D24
:10050000822A5F2C8E2A11303902031C8E2A031D89
:100510008D2A95303802031C8E2A5F2C552A4130D3
:100520003A02031C942A5F2CBA0AB908031D9C2ABC
:1005300065303802031C9D2A4916491CD12A3A0805
:10054000B100B2010310B10DB20DB10DB20DB10D7C
:10055000B20D3108A6003208A7004130A800A90159
:10056000D320BC008030A100212046305A206F30BB
:100570005A2075305A206E305A2064305A2020306C
:100580005A2073305A2069305A20C03021206730F9
:100590005A206E305A2061305A206C305A20203058
:1005A0005A203C2A491CF22A012049305A206E3038
:1005B0005A2069305A2074305A2069305A206130EC
:1005C0005A206C305A2069305A208030A100C03047
:1005D00021207A305A2065305A202E305A205A2055
:1005E0005A20552B0130BC000230A2003C080B20E1
:1005F000A101C91D0A2B3B3040020318012BC00A80
:10060000092BC001173044020318082BC40A092B18
:10061000C4010E2B4108C0004508C4001D2BC408AE
:10062000031D152B0C30C6001C2B0D304402031C7F
:100630001C2B0C304402C6001F2B4408C6000A3095
:1006400046020318252B20305A208030A10046088E
:1006500028203A305A200230A400400829203A309D
:100660005A2030305A205A20412B0C3044020318B3
:100670003C2B61305A203E2B70305A200630BC0093
:10068000432B0730BC000130C008031D0030B5000B
:100690001E3040020130031D0030B50401308618C1
:1006A0000301B5040319552B382C491E362CE821BB
:1006B0000130C8000F3048020318622BE821C80A35
:1006C000031D5A2B4911C911E821E821E821C91C51
:1006D0006B2B05146C2B05101230C8001430480227
:1006E0000318762BE821C80A031D6E2BE82107307A
:1006F000BB00AD214208C100E821491D802BC9156E
:100700000630BB00AD214208C500E821491D892BF8
:10071000C9150630BB00AD214208BD000330BB0047
:10072000AD214208C7000530BB00AD214208BF0023
:100730000830BB00AD214208BE00E821491DA12BB5
:10074000C915491CA72BC919A62B49100120C91985
:10075000352C8030A10021203D08282020305A204F
:1007600001303F02031DBB2B4A305A2061305A2012
:100770006E305A20332C02303F02031DC62B463008
:100780005A2065305A2062305A20332C03303F0201
:10079000031DD12B4D305A2061305A2072305A201F
:1007A000332C04303F02031DDC2B41305A207030C3
:1007B0005A2072305A20332C05303F02031DE72B9C
:1007C0004D305A2061305A2079305A20332C06306F
:1007D0003F02031DF22B4A305A2075305A206E30EA
:1007E0005A20332C07303F02031DFD2B4A305A207C
:1007F00075305A206C305A20332C08303F02031DCC
:10080000082C41305A2075305A2067305A20332C3A
:1008100009303F02031D132C53305A2065305A20F3
:1008200070305A20332C0A303F02031D1E2C4F30EB
:100830005A2063305A2074305A20332C0B303F0238
:10084000031D292C4E305A206F305A2076305A2002
:10085000332C0C303F02031D332C44305A206530BA
:100860005A2063305A2020305A20372C5F2C392AE6
:10087000851F3F2C8316051283120512412C831607
:10088000051683129B30B1200130C008031D0030D3
:10089000B500013086180301B5040319502C051565
:1008A000851585140130A900F430B2200511851199
:1008B00085100130A9004A30B220C30A582B01200C
:1008C0004E305A206F305A2020305A2073305A2030
:1008D00069305A2067305A206E305A2061305A20D1
:1008E0008030A100C03021206C305A20203084009C
:1008F0006030AB20A03084005030AB20203084002A
:100900003030AA208310061883148318C916831C5C
:10091000C91203010618013EC91A013C031D962C99
:10092000B60A0319B70A0130B120892C0301C91A8C
:100930000130013A0319C912031DC9160301061833
:10094000013EC91A013C031DAB2CB60A0319B70AB4
:100950000130B1209E2C03303702DE3003193602FD
:0A0960000318762C4914392AB42C30
:02400E00503F21
:00000001FF
